:020000040000FA
:060000000219FD02031CC1
:03000B0002008D63
:03001300020537AC
:03001B0002009050
:03002B000202D1FD
:03005B0002054655
:030073000203097C
:100080000406080C10182030406080A0C0054032E3
:10009000C2AFC2A853E6EFC28E856B8BC0D0D2D35D
:1000A000C0E0C0F0C2CAA8CCA9CDD2CAD2AF758A6E
:1000B00000C3E8956CF8E9956DF9C3E913F9E81305
:1000C000F8E5666007C3E913F9E813F8E97025E875
:1000D000956E4020956E501CE582B410177C007B15
:1000E000007A007908900000A86AE5667004C3E809
:1000F00013F801FD900000D2A8D2AA61E7E0FDC389
:100100009CC39840EF98EB33FB0582E0FCC39DC392
:100110009840E198EB33FB0582E0FDC39CC3984017
:10012000D398EB33FB0582E0FCC39DC39840C59890
:10013000EB33FB0582E0FDC39CC39840B798EB33DB
:10014000FB0582E0FCC39DC39840A998EB33FB05F7
:1001500082E0FDC39CC398409B98EB33FB0582E093
:10016000FCC39DC398408D98EB33FB0582217890AA
:100170000000D2A8D2AA61E7E0FDC39CC39840EF7B
:1001800098EA33FA0582E0FCC39DC39840E198EAFF
:1001900033FA0582E0FDC39CC39840D398EA33FA52
:1001A0000582E0FCC39DC39840C598EA33FA0582F6
:1001B000E0FDC39CC39840B798EA33FA0582E0FC9F
:1001C000C39DC39840A998EA33FA0582E0FDC39C19
:1001D000C398409B98EA33FA0582E0FCC39DC3981C
:1001E000408D98EA33FA0582EBC46B6A54F0F9EA61
:1001F000C454F0C3996009900000D2A8D2AA61E764
:10020000EBF4C454F0F9EAF4C4540F49FAEBF4C423
:10021000540FFBC3EAF99460FAEB9400FB5020C33F
:10022000E97B007A0079006016C3135006F9C39584
:1002300052600AE9F5527553007900800205533087
:100240003A27C3EA94D0F8EB9407F9400BE8FAE9AF
:10025000FB203509D235415D303502C235203902E7
:10026000B235C3EA33FAEB33FBEB2B3B3BF9C3EB81
:1002700013FBEA13FAEA29FAEB3400FB30E3047AC1
:10028000FF7BFFE5255403601B202A18E55D33F949
:10029000EB7007C3E99A4002E9FAE53CC4332AFA55
:1002A000EB3400FBC3EA33C4540FF8EB33C454F00F
:1002B00048F87005EA60027801900000D2A8D2AA3E
:1002C000E5226002152281D4900000D2A8D2AA6152
:1002D000E7C0D0C0E0C2CF0541E5666009E56560D2
:1002E000057565006104756501E52360021523C38A
:1002F000E55460057555006104E5552401F5555038
:10030000037555FFD0E0D0D032C2AF53E67F75926F
:10031000FA7593FFC22053917FD2AF32C0E0E58AD5
:10032000303408856B8BF0A3D0E032D0E0C2AF53FD
:10033000E6EFC0D0C0E0C0F0D2D3D2AF5388EFA870
:100340008AA98CAA40308D010A758A00758C0075C7
:100350004000438810E566700AC3E833F8E933F9D2
:10036000EA33FA30331FE8C4540FFAE9C454F04AB0
:10037000FAC3132AFAC3E833F8E933F9E82AFAE9A9
:100380003406FB61D830320FC3E833E933FAE82A88
:10039000FAE93400FB61D8303115E875F056A4AAAB
:1003A000F0E975F056A42AFAC5F03400FB61D8C311
:1003B000EA13FAE913F9E813F8E875F056A4AAF07D
:1003C000E975F056A42AFAC5F03400C313FBEA130A
:1003D000FAC3EB13FBEA13FAC3EB94125009C3EA16
:1003E0009434EB940750160522E52270021522C3BF
:1003F000E52294325002A12A755400A12DE5226015
:100400000215223036067C007D088117AC31AD32F2
:10041000303A04AC33AD34C3EA9CFAEB9DFB92084E
:10042000AE60AF61303A425007203509D235813590
:10043000303502C235303504AE62AF63203902B2C6
:1004400035C3EA33FAEB33FBA208500AEAF424017D
:10045000FAEBF43400FBC3EA9450FAEB9400FB503F
:100460001478007A007B008175A208500878007A21
:10047000007B0081D4E5255403601B202A18E55D2C
:1004800033F9EB7007C3E99A4002E9FAE53CC4335B
:100490002AFAEB3400FBEA8EF0A4F9AAF0EB8EF016
:1004A000A42AFAC5F03400FBC3EB13FDEA13F8C32A
:1004B000ED13FDE813F80FEF146004C3E833F8C33D
:1004C000E933EA33FAEB33FBDFEDEB30E30678FF99
:1004D0007AFF7B078854D230E86003755500C3E586
:1004E0005BFC955C4002AC5CC3EC95545008EC7529
:1004F000F008A4FAABF0EAF4F8EBF45407F98856E4
:10050000895775230AE55A30E210D0F0D0E0D0D0F8
:1005100053F7DF43F74043E61032D0F0D0E0D0D0BD
:1005200053D8FE43DA0143E6103275230AD0F0D0E7
:10053000E0D0D043E61032C2AAD28EC2CA85CC6CBB
:1005400085CD6DD2CA32C2AFC0D0C0E0D2D38556FD
:10055000FB8557FC85575A53F7BF53DAFED2A830B4
:100560003402D2AA53E6EF53F7DF53D8FED0E0D0DF
:10057000D0D2AF327901801479038010790A800CCF
:10058000791E80087964800479C880007817E4D5E2
:10059000E0FDD8FAD9F62278FF20282879A1E76073
:1005A00023E548601F74FF8548F084853FF03029BB
:1005B0000375F005A4F8C5F0600278FFC3E8955D07
:1005C0005002A85D885C22C3E54794A0E5489400EA
:1005D000E55C500314A1D8046002F55C2275E89034
:1005E00022055EC3E55E9408405330EDF4A8BDA932
:1005F000BE755E00E9FA79A0E76041EA7006E55F42
:100600006018800CC3E8955F600EE55F5005600AD6
:100610001480070460FA8002E55FF55FC3956940C6
:100620001B755BC0C394044013755B80C394044086
:100630000B755B40C394044003755B0022E55B24AB
:1006400010500274FFF55B22743279A687F0A4C5BE
:10065000F0A2F733F55D227547007548F022C2AF6E
:10066000C2CAA8CCA9CDAA4130CF010AD2CAD2AF02
:10067000C3EA13FAE913F9E813F8AB42AC43884232
:100680008943C3E89BF8E99C20280A547FF9302C61
:1006900002E17CC1D5AD448A44F9EA9D547FFA60F9
:1006A0000678FF79FFC1BAAE45AF468B458C46A8A8
:1006B00042A943C3E89EF8E99FF9C3E54813FBE567
:1006C0004713FAE82AF547E93BF54850067547FF16
:1006D0007548FFE122AA47AB48AC47AD487E047F8E
:1006E00002C3EB9404400D1E1FC3EB940840052089
:1006F00029021E1FC3ED13FDEC13FCDEF7C3EA9CB9
:10070000FAEB9DFBEF6009C3E913F9E813F8DFF793
:10071000EA28FAEB39FB8A478B4850067BFF8B4768
:100720008B48C3EB94025002D22C3028047F03E1A3
:100730004D7892E6FFC3E53D948240110FC3E53D3D
:1007400094A040010FC3EF940640027F057E02E5AE
:1007500048C4540FF9E548C454F0F8E547C4540FB1
:1007600028F8C3E89EFAE99400FB4009C3EA940123
:10077000EB940050047A01E4FB0207C8AA47AB4897
:10078000EBC4FEEAC4540F4EFCC3EA9CFAEB94009F
:10079000FBC3E813C313F8EA28FAEB3400FB8A47DB
:1007A0008B48C3EB94024002C22C7802EBC4FE7B60
:1007B00000EAC4540F4EFAC3EA98FA4005C3940104
:1007C00050027A017892E6FF302002E1C8854E920D
:1007D000854F93D22043E680C3E49AF8E49BF9C3A3
:1007E000E833F8E933F9302C0302085DE8FAE9FB55
:1007F000D3E913FDE813FC884E894FC3EF940360DF
:1008000038EF20E00CE82CF8E93DF9ECFAEDFB803C
:1008100013E828F8E939F9C3E82401F8E93400F9C4
:100820007AFF7BFFC3EF9403400F8A508B51884AB5
:10083000894B8C4C8D4D020892885089518A4A8B85
:100840004B8C4C8D4D3028127550F07551FF754C06
:10085000F0754DFF754EF0754FFF020892E8FAD320
:10086000E813FC884EC3EF94036021EF20E007E813
:100870002CF8ECFA017DE8282401F87AFFC3EF9404
:100880000340098A50884A8C4C02089288508A4A50
:100890008C4C3020020192753A02D22043E680E56A
:1008A000255403602DA847A948C3E913F9E813F8B4
:1008B000302804E92440F9C2AF53E67F759100C3A4
:1008C000E498F594E499F595759104D22043E68077
:1008D000D2AF22D221754900752000302B0375203C
:1008E0004001F1D221754900752040302B0375205D
:1008F0000078017901202C20E52554036002C221F3
:100900007914E548C313700104F8C39414400278C5
:1009100014302804781B791BC3E833F8C3E933F992
:10092000202010E549600C302803D53A04D222215A
:10093000A4119A0549E59B5440B52002218E302828
:100940000908C3E899400118212020210A08C3E8BA
:1009500099400201F12120C22153E67F75910030B8
:100960002C117594007595F0759104D22043E680A2
:100970000208F1E5487EFFC3334009C3334005C395
:10098000334001FEC3E49E759400F5952168C3E5EC
:10099000399401500201F130210201F1D80221A263
:1009A0002120C222C2AF53E67F7591008550948505
:1009B0005195759104854A92854B93D22043E680E8
:1009C000D2AFE52554036007202902053980103095
:1009D000220D202B0A202107158115810213F222F6
:1009E00078003021027801E53D75F007A4F9E5F0C3
:1009F00028F5F0E9A2F013A2F113A2F213F53DC31A
:100A000094785003753D78C3E53D953E4009C29307
:100A1000C294C29575D57F3020024117854C9285CE
:100A20004D93D22043E68022203814C2AFC294C234
:100A300090D293D29575D53BD2AF759F236128C2D2
:100A4000AFC294C292D295D29375D53ED2AF759F64
:100A5000236128203814C2AFC295D29475D53DC207
:100A600090D293D2AF759F136128C2AFC293D29434
:100A700075D53DC292D295D2AF759F0361282038BB
:100A800014C2AFC293C292D295D29475D53DD2AF63
:100A9000759F036128C2AFC295C290D293D294755C
:100AA000D53DD2AF759F136128203814C2AFC294D0
:100AB000D29375D53EC292D295D2AF759F238068EE
:100AC000C2AFC294D29575D53BC290D293D2AF75C6
:100AD0009F238054203814C2AFC295C291D294D2C1
:100AE0009375D53ED2AF759F13803DC2AFC293C2FE
:100AF00091D294D29575D53BD2AF759F03802920B2
:100B00003814C2AFC293D29575D53BC291D294D25C
:100B1000AF759F038012C2AFC295D29375D53EC206
:100B200091D294D2AF759F13227A147B7880127A77
:100B3000107B8C800C7A0D7BB480067A0B7BC8808E
:100B400000E564D5E001227902E4C294D5E0FDD24B
:100B500091D294D5E0FDC294D5E0FDC291D294D556
:100B6000E0FDE920E004D290D29330E004D292D2AA
:100B700095E564D5E0FDE920E002C29330E002C2D1
:100B8000957496D5E0FDD9C1EAF8D5E0FDD8FBDB38
:100B9000B0C29422C293C294C295C293C294C29529
:100BA00075D57F22788076FF0876FF0876FF087675
:100BB000FF0876FF0876FF0876090876FF087601B9
:100BC000788C76010876FF0876FF0876FF0876FFB6
:100BD0000876FF0876030876FF0876FF0876FF0898
:100BE00076250876D00876280876500876040876A8
:100BF000FF0876020876FF08767A0876FF087607FF
:100C00000876010876FF0876FF087600087600224D
:100C1000FA75F00CA4ABF0EAC333F8740133F9E8C9
:100C2000C333F8E933F9E8C32BF8E93400F9E8C332
:100C300033F8E933F9227888E6C39403D23A5002B4
:100C4000C23AC238E630E102D238A2389239788608
:100C5000E6149000809378A6F67886E6F53FC39474
:100C6000025003753F02789CE6753EFFB40203759F
:100C70003EA0B40303753E8278A0E6F860067428AF
:100C80002409D8FCF5697896E69110883189327884
:100C90009EE69110883389347897E69110883589DB
:100CA000367194223036117A007B007CFF7D007E05
:100CB00000B10A8B618A6022303A227896E6FA7B8C
:100CC00000789EE6FC7D00C3EA33FAEB33FBC3EC0D
:100CD00033FCED33FD7E0AB10A8B638A627896306D
:100CE0003A02789EE6FA7B007897E6FC7D007E006B
:100CF000303A10C3EA33FAEB33FBC3EC33FCED3389
:100D0000FD7E0AB10A8B618A6022C3EC9EFCED94E1
:100D100000FDC3EC9AFCED9BFDC3EC9423ED940025
:100D200050047C237D00C3EC94FFED940140047CCF
:100D3000FF7D017BFF0B7A000AEA7009C3EC33FCEC
:100D4000ED33FDA135EC8AF0A4AEF0ED8AF0A42ECF
:100D5000947C40E4EAF460DD22D23691A41205804E
:100D60001205807A007B007C10120578E5542AFA7F
:100D700074003BFBDCF37C04C3EB13FBEA13FADCEB
:100D8000F7FFEB60027FFFC23691A42278A5E6F957
:100D90005403C2857002D285E9540CC2867002D217
:100DA00086E95430C2877002D287E954C0700022AD
:100DB0007567007568007597DE7597AD7581C043DE
:100DC000FF8075EF0675A90071947580FF75F1F0CD
:100DD00075A4E07580FF75D4FF75900075F23F75BE
:100DE000A53F75900075D53F75A60175E34075E286
:100DF000027194E4F8F6D8FD71A412143C78988638
:100E000064753001C2AF1205887129120580712FF7
:100E10001205807135120580B18CC2AF75670075FF
:100E2000680078FA79FA308407D9FBD8F7021C00F9
:100E3000913691A478988664719475A91375A7105A
:100E400075C10075A70075660075E4047588117595
:100E50008E0475890975C80475910475D84075D9D3
:100E60000875F783759E0075960275DA4A75DB0082
:100E700075A82375E69075B801759B80759D007502
:100E8000D10C75BCB975BB1075E88075B20112053F
:100E900074D2AF753C00C230120588C231C232C272
:100EA00033C234755200755300752200120584C395
:100EB000E522940A5002E180D231752200120584A5
:100EC000C3E522940A5002E180C231D23275220079
:100ED000120584C3E522940A5002E18075E4C475CA
:100EE0008851758E017589AA758C00758D00C2A90F
:100EF000D2ABD2AA756B80756A14756E50C232D2AD
:100F00003475220A120584756A10C3E522940A75A5
:100F100052007553004069758E0C756B00756A2818
:100F2000756E2875220A120584756A20C3E522941D
:100F30000A7552007553004047758E0C756B8075AD
:100F40006A14756E1475220A120584756A10C3E559
:100F500022940A755200755300402575E404758883
:100F600011758E04758909D2A9C2ABC2AAC234D246
:100F700033752200120584C3E522940A4002C11A87
:100F8000120578203003020E1AC2AF71297129713F
:100F900029D2AF120588203403303A0302104212DE
:100FA0000578788CE6C394015003021042E530C303
:100FB000940150030210427567A57568F17F02D253
:100FC0003691A4120584C2AFC23691A4C3E55494ED
:100FD0007FD2AF406D120574C2AF713BD2AFDFDF7D
:100FE000B159C3EF7897F61205881215297F0AD2F6
:100FF0003691A4120584C2AFC23691A4C3E55494BD
:101000007FD2AF50E8120574C2AF120B2912057CD3
:10101000120B29D2AFDFD8120D59EF24037896F6C0
:10102000F87997E7C394234003985006E82423787F
:1010300097F61205889183B158120584120CA40208
:101040000E1A756700756800120584C3E554940193
:101050004003020F96C2AF120B3B120B3B120B3B2D
:10106000D2AF120588753000E4F537F5380537E55D
:1010700037F4703F0538789AE678191460127832A0
:1010800014600D787D14600878FA146003753800D8
:10109000C3E53898401D120B941205741538753746
:1010A0000078998664C2AF120B3BD2AF7898866401
:1010B00012058412057CE5237003020E1AC3E55461
:1010C0009401500AC3E5529401501602106D1205A6
:1010D00084E5237003020E1A755200755300021244
:1010E00083C3E55294017017C2AF120B94789986AE
:1010F00064120B2978988664D2AF1205844175C3B7
:10110000E55294027017C2AF120B9478998664125C
:101110000B2F78988664D2AF1205844175C3E552CF
:1011200094037017C2AF120B9478998664120B3532
:1011300078988664D2AF1205844175C3E552940451
:101140007017C2AF120B9478998664120B3B789893
:101150008664D2AF1205844175C3E55294057017B9
:10116000C2AF120B9478998664120B3B7898866410
:10117000D2AF1205844175C3E55294077019C3E5D7
:10118000539406500201BD7401303A02740378880A
:10119000F6C238C2394175C3E55294087019C3E5E7
:1011A000539406500201BD7402303A0274047888E8
:1011B000F6D238D2394175C3E55294097017C3E5A8
:1011C000539406500201BD303A0BC37888E694026E
:1011D000F6C23A4175C3E552940A7016C3E55394BA
:1011E00006500201BD203A0A7888E62402F6D23A77
:1011F0004175C3E55294147025C3E553940650021B
:1012000001BDC2AF901A0B740093D2AF7888F61369
:10121000C238C2394002D2384002D2398057C3E5C1
:101220005294157038C3E5539406404FC2AF901ADC
:101230000B740093D2AFF8B801027402B8020274C2
:1012400001B803027404B8040274037888F613C268
:1012500038C2394002D2384002D2398018C3E55230
:10126000940C70117567A57568F1C3E55394064039
:101270000A9183D2AF755200755300756700756887
:101280000001BDC2AF120B94E4D2AFE4F55EF524C9
:10129000F525F53D755E081205741205DD30EDFD8E
:1012A000A8BDA9BEE97001F8885F1205E1755E0866
:1012B000C2AF120648855D5B855D5CD2AF75A71035
:1012C00075C13075A70075A903756601303A07C26C
:1012D00038303502D238D228753900120AD4120AB1
:1012E000FF12065712065E12065712065E120657C6
:1012F0001208E31209E0120A2812065E1208D3202F
:101300002C03120597302C031205C71209E0120AAC
:101310005312065E1208E31209E0120A7E12065EFC
:101320001208D31209E0120AA912065E1208E3128B
:1013300009E0120AD412065E1205DD1208D3120962
:10134000E0120AFF1205E112065E302827855D5B78
:1013500079187A0CC3E53999400EC228D2298A3B04
:10136000855D5B855D5C800CC3E5549401400302A0
:1013700012F061FA30291F202B1CE53B147006C2C5
:1013800029D22A41F0F53B203A07C3E554940140A5
:10139000030212F08064753C00203A0F78FA79A4B9
:1013A000E760027803C3E55598504FE523604B3062
:1013B0003A17203805203507800F303502800A2083
:1013C0002B07D22B855D5B612078F0302B05855D86
:1013D0005B7820C3E5489850030212F0302B1BC203
:1013E0002BC238303502D238D229753B12855D5B6D
:1013F00041F0053CE554600261FD753C00C2AF124E
:101400000B9475240075250075A91375A71075C177
:101410000075A700756600D2AF120584120B947890
:10142000A4E6600CC290D293C291D294C292D2959B
:10143000C3E53C94044003020E1A0168901A0D782B
:101440002091BCE520B4550AA391BCE520B4AA02C2
:1014500080137567A57568F1120BA49183756700F9
:10146000756800801D901A0378807B0A91BCA308E0
:10147000DBFA901A0F788C7B1A91BCA308DBFA90E8
:101480001A2922C2AF91FF91DC901A00741091C109
:10149000A3740791C1A3742191C1901A0378807B32
:1014A0000A91C0A308DBFA901A0F788C7B1A91C0BE
:1014B000A308DBFAB11291F0901A2922E493F622E4
:1014C000E6438F01538FFDFFC3E583941C40012247
:1014D000EF8567B78568B7F0538FFE22438F0243CD
:1014E0008F018567B78568B7901A0DF0538FFC227E
:1014F000901A0D745591C1901A0E74AA91C1227A56
:101500003079D07820901A4091BCE520F709A3DA11
:10151000F7227A3079D0901A40E791C109A3DAF91D
:10152000227C05120588DCFB22C2AF120B29120BAC
:101530002F120B35120B3B12057C120B29120B2FAD
:10154000120B35120B3B12057C120B29120B2F12BA
:101550000B35120B3BD2AF22C2AF120B3B120B3535
:10156000120B2F120B2912057C120B3B120B35129A
:101570000B2F120B2912057C120B3B120B35120B91
:071580002F120B29D2AF224C
:1019FD00020DB0100721FFFFFFFFFFFF09FF01FFE1
:101A0D0055AA01FFFFFFFFFF03FFFFFF25D0285061
:0D1A1D0004FF02FF7AFF0701FFFF0000FF3A
:101A4000234A5F485F3030232020202020202020A0
:101A500023424C48454C492445464D3842323123B7
:101A60002020202020202020202020202020202076
:101C0000C2AFC2D37597DE7597AD7581C075A90057
:101C100043FF80752438752503B1DB7529A5752A26
:101C2000F143F11053A4EFD28475D4FF75E3407DE6
:101C3000FA780379E67C10752200752300901DE880
:101C40007B0675249875250130840281482084081C
:101C5000D8FBD9F9DCF781BA308408D8FBD9F9DC94
:101C6000F781BAB19BE493A3C39A6004DDC381BA40
:101C7000DBDBB18D600281317B08E493FAA3B16EA6
:101C8000DBF87A30B16E752200752300B18DEAFC65
:101C9000EBFDC3ED94FE400EB18D8A278B28ED300D
:101CA000E0048A828B83B18D7AC270D8C3ED94FE32
:101CB000601950CEBD0029EC600F7520007521FF22
:101CC000752900752A000200008100A827A92808AC
:101CD00009D804D90281DDB191EAF281D10D81A642
:101CE000C3ED94035051EDA2E092007AC5C3E582A2
:101CF0009400E583941C508C200010438F02438F86
:101D0000018529B7852AB7F0300027A827A9280818
:101D100009438F01538FFDD804D902A132C3E58353
:101D2000941C4003A3A117E28529B7852AB7F0A325
:101D3000A117538FFC81827AC1BD030CE493A3FAEF
:101D4000B152DCF8B14A81828184AA22AB23B16E00
:101D5000EBFAEA6222752608C3E52313F523E52290
:101D600013F52250066323A0632201D526EAB1DBD6
:101D7000B1DB75260AEAF4200102D284300102C2E6
:101D800084B1DBC3134002C201D526EB22B191EA34
:101D9000FB208402A191308402A196752608AE240E
:101DA000AF25C3EF13FFEE13FEB1DFB1DBC3EA13C0
:101DB0003084024480FA30E703632201C3E5231331
:101DC000F523E52213F52250066323A0632201D5F3
:101DD00026D9E52265236523F52222AE24AF250E00
:101DE0000FDEFEDFFCD20122424C48656C693437BD
:061DF0003164E8B20601B7
:00000001FF
